:100000003AC100002CC7000001C70000D6C600009E
:10001000ABC6000080C6000055C600005CC10000F1
:100020005AC1000058C1000056C1000054C1000070
:1000300052C1000050C100004EC100004CC1000080
:100040004AC1000048C1000046C1000044C1000090
:1000500042C1000040C100003EC10000E9C50000EF
:100060003AC10000AFC5000084C5000034C10000E3
:1000700032C1000030C100002EC100002CC10000C0
:100080002AC1000028C1000026C1000024C10000D0
:1000900022C1000020C100001EC100001CC10000E0
:1000A0001AC1000018C1000016C1000014C10000F0
:1000B00012C1000010C100000EC100000CC1000000
:1000C0000AC1000008C1000006C1000004C1000010
:1000D00002C1000000C10000FEC00000FCC0000022
:1000E000FAC000002F0A002300230023005C232312
:1000F00023235265616C53696D476561722300006B
:100100000020002300260029002C002F00320000D0
:10011000010000030106010901000021002400275D
:10012000002A002D00300033000101000004010707
:10013000010A0100002200250028002B002E0031BA
:1001400000340002010000050108010B010505054E
:1001500005070508080808020202020A0A0808043E
:10016000040404010101010101010103030303036C
:10017000030303040707070C0C0C0C0C0C0C0C02FB
:1001800002020206060606060606060B0B0B0B0B02
:100190000B0B0B01021020200808102040102040FB
:1001A000800201020108040201010204081020403B
:1001B0008080402010080402018004020180402059
:1001C0001008040201080402010102040810204082
:1001D00080010204081020408000000A0B02090C74
:1001E0000D0E0807030401000000000000000000DD
:1001F00000000000000000000000000000000000FF
:1002000000000000001211100000000000000000BB
:100210000000000000000000000000000000002FAF
:100220000A002300230023005C232323235265615B
:100230006C53696D4765617223000A000A003D0036
:100240000A003D003D300A002E4F46460A003D316F
:100250000A002E4F4E0A002F0A002300230023001D
:100260005C232323235265616C53696D476561727A
:1002700023005807FD0A11241FBECFEFD1E2DEBFD5
:10028000CDBF00E00CBF2AE0AAEAB5E001C01D9294
:10029000A930B207E1F715E0A0E0B2E0EEE2FBE141
:1002A00000E00BBF02C007900D92AA3AB107D9F740
:1002B00011E0CAE3D1E000E006C021970109802FD8
:1002C000FE010E944B0BC933D10780E00807A9F754
:1002D00071D60C94860D94CEAF92BF92CF92DF92DE
:1002E000EF92FF920F931F93CF93DF936C017B01EB
:1002F0008B01040F151FEB015E01AE18BF08C0177C
:10030000D10759F06991D601ED91FC910190F081EE
:10031000E02DC6011995892B79F7C501DF91CF91A1
:100320001F910F91FF90EF90DF90CF90BF90AF9013
:100330000895E3ECF6E044815581608171818DE19F
:1003400096E0CACFFC01538D448D252F30E0842FD9
:1003500090E0821B930B541710F0CF9608950197ED
:100360000895FC01918D828D981761F0A28DAE0FDA
:10037000BF2FB11D5D968C91928D9F5F9F73928F61
:1003800090E008958FEF9FEF0895FC01918D828D8D
:10039000981731F0828DE80FF11D858D90E008955A
:1003A0008FEF9FEF0895FC01918D228D892F90E0B2
:1003B000805C9F4F821B91098F73992708958DE16F
:1003C00096E0F1DF21E0892B09F420E0822F0895E7
:1003D000FC01A48DA80FB92FB11DA35ABF4F2C91BA
:1003E000848D90E001968F739927848FA689B789B1
:1003F0002C93A089B1898C91837080648C93938DA8
:10040000848D981306C00288F389E02D80818F7D4A
:1004100080830895EF92FF920F931F93CF93DF9302
:10042000EC0181E0888F9B8D8C8D98131AC0E88930
:10043000F989808185FF15C09FB7F894EE89FF89FF
:100440006083E889F98980818370806480839FBF9D
:1004500081E090E0DF91CF911F910F91FF90EF909D
:100460000895F62E0B8D10E00F5F1F4F0F731127AD
:10047000E02E8C8D8E110BC00FB607FCFACFE889E9
:10048000F989808185FFF5CFCE01A2DFF2CFEB8D18
:10049000EC0FFD2FF11DE35AFF4FF0829FB7F89448
:1004A0000B8FEA89FB8980818062D0CF0F931F93E5
:1004B000CF93DF938C01D0E0C0E0F801EC0FFD1F7B
:1004C0006491662339F08DE196E0A4DF892B11F069
:1004D0002196F3CFCE01DF91CF911F910F91089517
:1004E000CF93DF93EC01888D8823B1F0AA89BB8973
:1004F000E889F9898C9185FD03C0808186FD0CC057
:100500000FB607FCF7CF8C9185FFF2CF808185FF76
:10051000EDCFCE015DDFEACFDF91CF91089581501D
:10052000823108F05AC0E82FF0E08827E556FD4FE9
:100530008F4F0C944B0BBB02BF02AD02B302B7024C
:10054000ED02C202C802CC02D202D602DA02E002F6
:10055000E402ED02E802EE02F202809180008F7761
:10056000809380000895809180008F7DF9CF8091E5
:100570008000877FF5CF84B58F7784BD089584B5DB
:100580008F7DFBCF8091B0008F778093B00008956E
:100590008091B0008F7DF9CF809190008F7780930C
:1005A00090000895809190008F7DF9CF8091900008
:1005B000877FF5CF8091A0008F778093A00008956A
:1005C0008091A0008F7DF9CF8091A000877FF5CF2B
:1005D000809120018F7780932001089580912001E0
:1005E0008F7DF9CF80912001877FF5CF1F93CF9327
:1005F000DF93282F30E0F901E752FE4F8491F90193
:10060000ED56FE4FD491F901E35BFE4FC491CC232C
:10061000A1F0162F811183DFEC2FF0E0EE0FFF1F0A
:10062000ED5CFE4FA591B4918FB7F894EC91111148
:1006300008C0D095DE23DC938FBFDF91CF911F914F
:100640000895DE2BF8CFCF93DF9390E0FC01ED56B9
:10065000FE4F2491835B9E4FFC0184918823C9F057
:1006600090E0880F991FFC01E75EFE4FA591B491C1
:10067000FC01ED5CFE4FC591D49161110DC09FB797
:10068000F8948C91209582238C9388812823288349
:100690009FBFDF91CF910895623051F49FB7F894D6
:1006A0003C91822F809583238C93E8812E2BEFCF72
:1006B0008FB7F894EC912E2B2C938FBFEACF863313
:1006C00008F0865320917B00982F9870277F922BFB
:1006D00090937B008770806480937C0080917A0087
:1006E000806480937A0080917A0086FDFCCF8091AF
:1006F00078009091790008953FB7F894809115069D
:1007000090911606A0911706B091180626B5A89BE1
:1007100005C02F3F19F00196A11DB11D3FBFBA2F93
:10072000A92F982F8827BC01CD01620F711D811D53
:10073000911D42E0660F771F881F991F4A95D1F7D8
:1007400008958F929F92AF92BF92CF92DF92EF92D5
:10075000FF924B015C01D0DF6B017C01CDDF6C1996
:100760007D098E099F09683E734081059105B0F3AC
:1007700021E0821A9108A108B10888EEC80E83E032
:10078000D81EE11CF11C81149104A104B10431F7BD
:10079000FF90EF90DF90CF90BF90AF909F908F90A1
:1007A00008952FB7F8946091110670911206809108
:1007B0001306909114062FBF0895862F642F43CF00
:1007C000CF93DF93FC01218530E0F901E752FE4F22
:1007D0008491F901ED56FE4FD491F901E35BFE4F90
:1007E000C491CC2371F081119ADEEC2FF0E0EE0F72
:1007F000FF1FE150FF4FA591B491EC91ED2381E0F3
:1008000009F480E08170DF91CF910895DC01ED91D2
:10081000FD918081ED91FD919081ED91FD916C9123
:1008200063708E2309F064609F2309F06860E3E23F
:10083000F4E0E60FF11D659565956D936D917D91E1
:100840008D919D91099423C01AC012C016C010C08A
:100850001EC009C014C013C006C019C009C00DC015
:1008600007C00DC014C062507040804090400BC063
:10087000615070408040904006C06E5F01C06F5F65
:100880007F4F8F4F9F4F9E938E937E936E930895CD
:100890008F929F92AF92BF920F931F93CF93DF934C
:1008A000CDB7DEB7A1970FB6F894DEBF0FBECDBFB0
:1008B00019A2423008F44AE08E010F5D1F4F842ECA
:1008C000912CB12CA12CA5019401C3D6E62FB9011E
:1008D000CA01EA303CF5E05DD801EE938D01232B8F
:1008E000242B252B81F790E080E0109761F0FD012B
:1008F00001900020E9F73197AF014A1B5B0BBD0166
:100900008DE196E0E9DCA1960FB6F894DEBF0FBE4C
:10091000CDBFDF91CF911F910F91BF90AF909F906E
:100920008F900895E95CD8CFCF92DF92EF92FF923B
:10093000CF93DF936C01990FEE08FF08F7FE17C005
:100940006DE28DE196E066DDEC0166277727CB014D
:100950006C197D098E099F094AE09ADF8C0F9D1F53
:10096000DF91CF91FF90EF90DF90CF9008954AE014
:10097000C701B601DF91CF91FF90EF90DF90CF904C
:1009800087CF009761F0FC0101900020E9F73197D3
:10099000AF01481B590BBC018DE196E09DCC90E066
:1009A00080E008950F931F93CF93DF938DE196E03E
:1009B000FADC892B09F450C08DE196E0D2DC8C374B
:1009C000D1F48DEE90E072DD8AEF92E0DADF8BEE0B
:1009D00090E06CDD87E090E0A7DF89EE90E066DDD7
:1009E00084E092E0CEDF87EE90E060DDA2DC84EE72
:1009F00090E05CDDDBCF8C3329F410920F0610926F
:100A00000E06D4CF8A30B1F4C4E1D2E00AEA15E090
:100A100089919991009739F0F801208161E02133A3
:100A200009F060E0E3DD0F5F1F4FF2E0C832DF073F
:100A300079F7E3CF20910E0630910F062436310569
:100A4000E4F6F901E655FA4F80832F5F3F4F30936C
:100A50000F0620930E06AACFDF91CF911F910F9121
:100A60000895ADDC81119EDF80E090E0892B49F094
:100A700080E090E0892B29F00E94000081110E9403
:100A8000000080E090E0892B49F080E090E0892B25
:100A900029F00E94000081110E94000080E090E097
:100AA000892B49F080E090E0892B29F00E9400001A
:100AB00081110C9400000895CF93DF93EC0188819D
:100AC0009981009709F08BD6198218821D821C82A9
:100AD0001B821A82DF91CF910895FC018081918160
:100AE000009709F07CC608950F931F93CF93DF936F
:100AF000EC0188819981009759F02A813B81261762
:100B0000370730F081E0DF91CF911F910F91089569
:100B10008B016F5F7F4FECD6009759F099838883E4
:100B20001B830A832C813D81232B61F7FC011082FA
:100B3000E9CF80E0E8CFEF92FF920F931F93CF931E
:100B4000DF93EC017B018A01BA01CEDF81110AC07B
:100B5000CE01B2DFCE01DF91CF911F910F91FF90B7
:100B6000EF9008951D830C83B70188819981ADD7DB
:100B7000F1CF1F920F920FB60F9211240BB60F9266
:100B80002F933F934F935F936F937F938F939F9395
:100B9000AF93BF93EF93FF938DE196E019DCFF9144
:100BA000EF91BF91AF919F918F917F916F915F91E5
:100BB0004F913F912F910F900BBE0F900FBE0F9052
:100BC0001F9018951F920F920FB60F9211240BB61B
:100BD0000F922F938F939F93EF93FF93E0912D06A6
:100BE000F0912E068081E0913306F091340682FD6B
:100BF0001DC09081809136068F5F8F7320913706DC
:100C0000821741F0E0913606F0E0E35EF94F958FF0
:100C100080933606FF91EF919F918F912F910F90C6
:100C20000BBE0F900FBE0F901F9018958081F2CFD2
:100C30001F920F920FB60F9211242F933F938F9311
:100C40009F93AF93BF938091110690911206A0914C
:100C50001306B09114063091100623E0230F2D37B0
:100C600058F50196A11DB11D209310068093110621
:100C700090931206A0931306B09314068091150664
:100C800090911606A0911706B09118060196A11D25
:100C9000B11D8093150690931606A0931706B09386
:100CA0001806BF91AF919F918F913F912F910F9017
:100CB0000FBE0F901F90189526E8230F0296A11DD6
:100CC000B11DD2CF1F920F920FB60F9211240BB607
:100CD0000F922F933F934F935F936F937F938F93D5
:100CE0009F93AF93BF93EF93FF9390E080E08EDDEF
:100CF000FF91EF91BF91AF919F918F917F916F91F4
:100D00005F914F913F912F910F900BBE0F900FBEAF
:100D10000F901F9018951F920F920FB60F921124EB
:100D20000BB60F922F933F934F935F936F937F93E5
:100D30008F939F93AF93BF93EF93FF9390E080E0E7
:100D400065DDFF91EF91BF91AF919F918F917F9161
:100D50006F915F914F913F912F910F900BBE0F902C
:100D60000FBE0F901F9018951F920F920FB60F9203
:100D700011240BB60F922F933F934F935F936F9372
:100D80007F938F939F93AF93BF93EF93FF9390E0E5
:100D900080E03CDDFF91EF91BF91AF919F918F91EA
:100DA0007F916F915F914F913F912F910F900BBE6B
:100DB0000F900FBE0F901F9018951F920F920FB6B5
:100DC0000F9211240BB60F922F933F934F935F9383
:100DD0006F937F938F939F93AF93BF93EF93FF9303
:100DE00090E080E013DDFF91EF91BF91AF919F9173
:100DF0008F917F916F915F914F913F912F910F90C4
:100E00000BBE0F900FBE0F901F9018951F920F9260
:100E10000FB60F9211240BB60F922F933F934F935F
:100E20005F936F937F938F939F93AF93BF93EF9352
:100E3000FF9390E080E0EADCFF91EF91BF91AF91EA
:100E40009F918F917F916F915F914F913F912F91E2
:100E50000F900BBE0F900FBE0F901F9018951F9212
:100E60000F920FB60F9211240BB60F922F933F9350
:100E70004F935F936F937F938F939F93AF93BF93A2
:100E8000EF93FF9390E080E0C1DCFF91EF91BF9181
:100E9000AF919F918F917F916F915F914F913F9112
:100EA0002F910F900BBE0F900FBE0F901F901895B3
:100EB0001092200610921F0688EE93E0A0E0B0E0AA
:100EC0008093210690932206A0932306B0932406D4
:100ED00084EE92E090931E0680931D0685EC90E0D0
:100EE00090932A068093290684EC90E090932C0638
:100EF00080932B0680EC90E090932E0680932D0635
:100F000081EC90E09093300680932F0682EC90E085
:100F1000909332068093310686EC90E090933406ED
:100F200080933306109236061092370610923806D8
:100F300010923906AAEBB6E090E080E041E2FC01B5
:100F40003E9621E030E08630910510F430E020E05C
:100F5000E20FF31F40935700E491ED93019689301F
:100F6000910569F7E9ECF6E026EF32E08AE090E0DF
:100F700031832083128213821482158297838683A1
:100F80001086118672964AE0E530F40789F71092D0
:100F9000C4061092C3061092C6061092C50610929F
:100FA000C8061092C70650E040E061E273E083ECAF
:100FB00096E0C1CDCF93DF93CDB7DEB72F970FB6B5
:100FC000F894DEBF0FBECDBF789484B5826084BD37
:100FD00084B5816084BD85B5826085BD85B581603D
:100FE00085BD80916E00816080936E0010928100BB
:100FF0008091810082608093810080918100816076
:101000008093810080918000816080938000809136
:10101000B10084608093B1008091B00081608093C2
:10102000B000809191008260809391008091910046
:101030008160809391008091900081608093900006
:101040008091A10082608093A1008091A1008160C5
:101050008093A1008091A00081608093A000809186
:101060002101826080932101809121018160809320
:1010700021018091200181608093200180917A007C
:10108000846080937A0080917A00826080937A00F5
:1010900080917A00816080937A0080917A008068E4
:1010A00080937A001092C100E0912D06F0912E06F7
:1010B00082E08083E0912906F0912A061082E09177
:1010C0002B06F0912C0680E1808310923506E0918A
:1010D0003106F091320686E08083E0912F06F09190
:1010E0003006808180618083E0912F06F091300688
:1010F000808188608083E0912F06F09130068081A6
:1011000080688083E0912F06F091300680818F7D8A
:10111000808382E390E0A0E0B0E08093210690938A
:101120002206A0932306B093240668EE73E080E0C5
:1011300090E007DB6BEBC62E66E0D62E8E010F5FCC
:101140001F4FD6018D916D011B861A861D861C8648
:101150001F861E8640E1B80190E052D2F80101904E
:101160000020E9F73197AF01401B510BB801CE01C8
:101170000A96E1DC1A8219821C821B821E821D8261
:101180006091C3067091C4066115710531F04091FC
:10119000C7065091C806C801CEDC8E859F85AA84FB
:1011A000BB84ED80FE80E80EF91EA114B10409F4A1
:1011B00039C0892B79F0B701C80196DC882391F1F9
:1011C00029813A818D819E81B501820F931F7DD443
:1011D000FE82ED8269817A816115710531F14D815F
:1011E0005E8183EC96E0A7DCC80177DCCE010A962D
:1011F00074DCB3ECCB16B6E0DB0609F0A2CF0091AD
:10120000C3061091C4060115110599F0F8018081FB
:10121000882379F0082E000C990B46D4D8018D93C1
:101220008D01F4CFC80148DCD5CF83EC96E044DCD7
:10123000DBCF88E292E03AD98AEF92E0A2DB86E245
:1012400092E034D987E090E06FDB84E292E02ED91F
:1012500084E092E096DB82E292E028D96AD88FE1BE
:1012600092E024D909EC16E048E2E42E42E0F42EA4
:101270005AE0A52EB12CF701D0807181D801ED91F3
:10128000FC910280F381E02D42E050E06D2DC80119
:101290001995F801D18610860190F081E02D01901A
:1012A000F081E02DC8011995882339F0D8011896EE
:1012B0008C911897836018968C9373DAF801628387
:1012C000738384839583B782A682F4E0EF0EF11CCA
:1012D0000E5E1F4F8AE00530180769F624E1E22E02
:1012E00022E0F22E38E2A32E32E0B32E8701D8019D
:1012F000CD90DD908D01C114D10431F061E08C2DD1
:10130000A2D961E08C2D72D9A016B10681F768EBE5
:101310007BE080E090E015DAF701819191917F0107
:10132000009711F060E062D90E151F05A9F7772428
:10133000739492E0692E35DA6B017C0180910A0288
:1013400090910B02A0910C02B0910D02AC01BD0175
:101350004854544F6F4F7F4FC416D506E606F70624
:1013600028F4C816D906EA06FB0650F580E692E096
:101370009DD88AEF92E005DB8EE592E097D887E072
:1013800090E0D2DA8CE592E091D884E092E0F9DA4C
:101390008AE592E08BD80E94990187E592E086D891
:1013A000C0920A02D0920B02E0920C02F0920D025F
:1013B000C0920002D0920102E0920202F092030277
:1013C00061E070E080E090E0BCD988E2A82E82E085
:1013D000B82E09EC16E0D80118968C9118978B7FDF
:1013E00018968C931897ED91FC910190F081E02D67
:1013F000C8011995982EF8018085869581709816F8
:1014000009F49EC0CED9D80112966D937D938D9329
:101410009C93159718968C911897862518968C93FF
:10142000D80118969C91892F847090FDCFC0882395
:1014300079F0F5018280938063EC74E0C4014CD3B1
:10144000892B09F4BEC0C4019CDA82E592E02ED853
:101450000E5E1F4FB4E0AB0EB11CEAE005301E0774
:1014600009F0B9CF86E32BD98C0180911B069091AE
:101470001C069C012F5031090217130724F00F9608
:101480008017910794F40B3011057CF010931C0623
:1014900000931B068EE093E074DA82E492E006D8B3
:1014A000C80142DA80E492E001D887E308D98C01D0
:1014B0008091190690911A069C012F50310902174C
:1014C000130724F00F9680179107A4F40B30110531
:1014D0008CF010931A060093190688E193E051DA14
:1014E0008EE392E00E945602C8011EDA8CE392E07D
:1014F0000E9456028091000290910102A091020286
:10150000B0910302AC01BD014C595F4F6F4F7F4F4B
:10151000C416D506E606F70628F4C816D906EA0664
:10152000FB0660F48AE392E00E945602C092000239
:10153000D0920102E0920202F092030292DAFBCE14
:1015400030D9F80122813381448155811B012C015E
:10155000221A330A440A550AB201A10186819781F1
:10156000B0E0A0E0481759076A077B0708F458CF96
:1015700080858170981609F453CF13D9D80112963B
:101580006D937D938D939C93159718968C911897D6
:101590008725846018968C9304D9F80122853385B9
:1015A00044855585621B730B840B950B6687778783
:1015B000808B918BF6D8F801628773878487958733
:1015C0002FCFC401DED98EE492E041CF882309F405
:1015D0003FCFD50112968D909C9063EC74E0C401CE
:1015E0007BD2892B29F0C401CCD988E492E02FCF9B
:1015F000C401C7D984E492E02ACF83EC96E06DCA97
:10160000BB27FB015527AA27880F991FAA1FA417DC
:1016100010F0A41B83955051B9F7A05DAA3308F0D0
:10162000A95DA193009779F7B111B1931192CB0104
:1016300000C0DC01FC01672F71917723E1F732973D
:1016400004C07C916D9370836291AE17BF07C8F39D
:101650000895A1E21A2EAA1BBB1BFD010DC0AA1FF3
:10166000BB1FEE1FFF1FA217B307E407F50720F00B
:10167000A21BB30BE40BF50B661F771F881F991F86
:101680001A9469F760957095809590959B01AC01CF
:10169000BD01CF010895EE0FFF1F881F8BBF07907C
:1016A000F691E02D19940F931F93CF93DF9382301F
:1016B000910510F482E090E0E091070AF091080AA9
:1016C00030E020E0B0E0A0E0309799F4211531053A
:1016D00009F44AC0281B390B24303105D8F58A811A
:1016E0009B816115710589F1FB0193838283FE0162
:1016F00011C0408151810281138148175907E0F0E0
:101700004817590799F4109761F012960C931297A5
:1017100013961C933296CF01DF91CF911F910F91B9
:1017200008950093070A1093080AF4CF2115310594
:1017300051F04217530738F0A901DB019A01BD01AE
:10174000DF01F801C1CFEF01F9CF9093080A809330
:10175000070ACDCFFE01E20FF31F81939193225030
:10176000310939832883D7CF2091050A3091060AA1
:10177000232B41F420911002309111023093060A7C
:101780002093050A20910E0230910F022115310598
:1017900041F42DB73EB74091120250911302241B21
:1017A000350BE091050AF091060AE217F307A0F461
:1017B0002E1B3F0B2817390778F0AC014E5F5F4FA7
:1017C0002417350748F04E0F5F1F5093060A4093C9
:1017D000050A819391939FCFF0E0E0E09CCFCF93F7
:1017E000DF930097E9F0FC01329713821282A091F7
:1017F000070AB091080AED0130E020E01097A1F44B
:1018000020813181820F931F2091050A3091060AB1
:101810002817390709F061C0F093060AE093050A1A
:10182000DF91CF910895EA01CE17DF07E8F54A81ED
:101830005B819E0141155105B1F7E901FB83EA8304
:1018400049915991C40FD51FEC17FD0761F48081B0
:1018500091810296840F951FE90199838883828183
:1018600093819B838A83F0E0E0E012968D919C91B6
:1018700013970097B9F52D913C911197CD010296E0
:10188000820F931F2091050A3091060A2817390705
:1018900039F6309751F51092080A1092070AB09362
:1018A000060AA093050ABCCFD383C283408151812D
:1018B000840F951FC817D90761F44E5F5F4F888169
:1018C0009981480F591F518340838A819B8193835B
:1018D00082832115310509F0B0CFF093080AE09317
:1018E000070A9ECFFD01DC01C0CF13821282D7CF41
:1018F0004F925F926F927F928F929F92AF92BF9220
:10190000CF92DF92EF92FF920F931F93CF93DF93CB
:101910008C01009791F4CB01DF91CF911F910F9132
:10192000FF90EF90DF90CF90BF90AF909F908F90FF
:101930007F906F905F904F90B6CEFC01E60FF71F3F
:101940009C0122503109E217F30708F4AAC0D9011B
:10195000CD91DC911197C617D70718F1C530D10585
:1019600070F0CE0104978617970748F0C61BD70B77
:101970002297C193D1936D937C93CF0130DFC8013F
:10198000DF91CF911F910F91FF90EF90DF90CF905B
:10199000BF90AF909F908F907F906F905F904F908F
:1019A00008955B01AC1ABD0A4C018C0E9D1EA091DE
:1019B000070AB091080A512C412CF12CE12C109708
:1019C00031F58091050A9091060A8815990509F06C
:1019D0005CC04616570608F058C080910E029091E0
:1019E0000F02009741F48DB79EB7409112025091BB
:1019F0001302841B950BE817F90708F052C0F09307
:101A0000060AE093050AF90171836083B8CF8D91CE
:101A10009C91119712966C90129713967C90139745
:101A2000A815B90559F56C0142E0C40ED11CCA14C1
:101A3000DB0420F1AC014A195B09DA011296159713
:101A400080F06282738251834083D9016D937C93CD
:101A5000E114F10471F0D7011396FC93EE93129701
:101A60008ECF22968C0F9D1FF90191838083F30105
:101A7000EFCFF093080AE093070A81CF4816590682
:101A800008F42C017D01D3019ACFCB010CDE7C013F
:101A9000009739F0AE01B8010FD0C801A0DE870170
:101AA0006ECF10E000E06BCF9111089581568A51FE
:101AB00008F4805285580895FB01DC0102C00190B2
:101AC0000D9241505040D8F70895FB01DC01019080
:101AD0000D920020E1F70895FB0151915523A9F0E3
:101AE000BF01DC014D9145174111E1F759F4CD01DA
:101AF0000190002049F04D9140154111C9F3FB01BF
:101B00004111EFCF81E090E00197089511E0CAE321
:101B1000D1E000E005C0802FFE01BDDD2196011D52
:0E1B2000CB33D10780E00807B1F7F894FFCF70
:101B2E00FFFFFFFF332E312E3900FFFFFFFF0000B6
:101B3E00090A80000E000F0009001E001F00080099
:101B4E001C001D00060007001300220310003203C4
:101B5E0022004203250052032D0062032B006F0367
:101B6E0029007C032A0088032E0094032C00A60370
:101B7E002800B8032600C4034200D0034400DE034D
:101B8E003E00EC034000F9032F000604300013045E
:101B9E00310023043200320433003F0434004D047C
:101BAE0035005D0402006B04030079040C00870409
:101BBE000A0095041A00A3041B00AF041100BB0415
:101BCE000B00C7040400D6040500E3041900F10459
:101BDE002300FD04210007054500140541002105E1
:101BEE003C002D053F0037053A004A0524005D05EF
:101BFE0027006E0520007805430083053D009605FD
:101C0E00000000000A026C01A2017002D301B101B2
:101C1E00C50100000000E003DD035265616C5369ED
:101C2E006D476561722D54424D2D504E4C00504FF4
:101C3E00545F50414E454C00504F545F4252414B01
:101C4E00450053575F4C44475F4C545F444E2E53F0
:101C5E00570053575F4C44475F4C545F55502E53BB
:101C6E00570053575F534F555243455F444E2E53C3
:101C7E00570053575F534F555243455F55502E53A0
:101C8E00570053575F47454E5F444E2E53570053F0
:101C9E00575F47454E5F55502E53570053575F536E
:101CAE00544152545F444E0053575F535441525463
:101CBE005F55500053575F49474E4954494F4E5F49
:101CCE00444E2E53570053575F49474E4954494F80
:101CDE004E5F55502E53570053575F42505F444E40
:101CEE002E53570053575F42505F55502E53570097
:101CFE0053575F5452494D5F444E2E53570053571E
:101D0E005F5452494D5F55502E53570053575F4500
:101D1E004C545F444E2E53570053575F454C545FFF
:101D2E0055502E53570053575F41465F4943452E3A
:101D3E0053570053575F4943455F4C494748542E0C
:101D4E0053570053575F50524F505F4943452E53E0
:101D5E00570053575F57535F4943452E5357005310
:101D6E00575F5049544F545F4C2E53570053575F93
:101D7E00494E4552545F5345502E53570053575FAB
:101D8E005049544F545F522E53570053575F474597
:101D9E0041525F55502E53570053575F474541529E
:101DAE005F444E2E53570053575F464C41505F448D
:101DBE004E2E53570053575F464C41505F55502E91
:101DCE0053570053575F41435F444E2E53570053B2
:101DDE00575F41435F55502E53570053575F424C48
:101DEE004545442E53570053575F50524553535554
:101DFE0052452E53570042544E5F43484B5F444F5B
:101E0E00574E0042544E5F43484B5F4C494748542F
:101E1E000053575F50554C53452E53570053575F41
:101E2E004E41562E53570053575F5354524F42450F
:101E3E002E53570053575F44494D4D45522E53571D
:101E4E000053575F434142494E2E53570053575F3D
:101E5E004143434553530042544E5F4D41494E5FFB
:101E6E0047454E5F52455345540042544E5F5354BE
:101E7E0042595F47454E5F52455345540053575F95
:101E8E004D41494E5F504F5745522E5357004254C5
:101E9E004E5F53484946540053575F4655454C2EA6
:101EAE0053570042544E5F4D41535445525F574174
:101EBE00524E494E470042544E5F4D415354455287
:0A1ECE005F43415554494F4E000098
:00000001FF
